:1000000000308A00A22E0000FF00030E8301A10031
:100010000A08A0008A010408A2007708A300780853
:10002000A4007908A5007A08A6007B08A70083131E
:1000300083128C308400001D1F280C1938288D3045
:100040008400001C25280D183B2822088400230862
:10005000F7002408F8002508F9002608FA00270808
:10006000FB0020088A00210E8300FF0E7F0E09008E
:100070008A110A123E288A110A124B28941314136B
:1000800094121430AB00C3010730BB0094160C115E
:100090008A110A12252870147008831687008312AB
:1000A00007185428031055280314B00CAF0CB208DD
:1000B00003195C28B20390280314AF0DB00D03148C
:1000C000AF0DB00D0A30B2003408F700F70803197D
:1000D0007A280130770203197D280230770203194C
:1000E000802803307702031983280430770203192C
:1000F000862889283008BC008A283008BD008A2854
:100100003008BE008A283008BF008A283008C000A6
:100110008A288A28B40A33083402031D9028B517A8
:100120000D108A110A122528733084000008031963
:10013000A6280630F800F701F70B9C28F80B9B283F
:100140007B30F700F70BA228800B99288A110A123E
:10015000A52983160D1073088312B300B401F501AD
:10016000F010700883168700831287103130F70073
:10017000F70BB82800000000701070088316870085
:10018000831207103130F700F70BC428000000007D
:10019000F0147008831687008312F0147008831619
:1001A000870083128718CD28F4017408073C031CCC
:1001B00003297208F7007408F8000319E3280310F4
:1001C000F70CF80BDF28771CED28701470088316E5
:1001D00087000130F5068312F3287010700883162B
:1001E000870083120710F0147008831687008312AB
:1001F000871CF328F0147008831687008312871871
:10020000FA28F40AD528F0147008831687008312A0
:1002100087180329F508031D132970147008831625
:1002200087008312192970107008831687008312C3
:100230000710F0147008831687008312871C192991
:100240001030F700F70B2229000070147008831695
:1002500087008312F01470088316870083128718B2
:100260002A29F0147008831687008312871C31290D
:1002700070147008831687008312071C422901300E
:10028000F6004329F601F0147008831687008312E4
:10029000871843290D1083160D1483120034B51FDF
:1002A0004F29B501B40100343F3085008601FF308D
:1002B000870088018901203083168500FF30860081
:1002C0001F308700F000FF308800091089100911E5
:1002D000811383121F0838399F00063083169F0050
:1002E00083129412F012700883168700701670083B
:1002F00087008516F015700887003430831294004B
:10030000003083169400831207119701053097007F
:1003100087109D0104309D008530900083160D14D8
:10032000C03083128B04AE01FF30AF00FF30B0004D
:100330000A30B200B501B401C301A801A901AA01A4
:100340000230F200FA30F3009428F20BA229FF30B9
:10035000F2000330F300A9204F21FF30F2000330F8
:10036000F300A9204F21FF30F2000330F300A92051
:100370004F21F230F2000230F300A9204F21E93082
:10038000F2000330F300A9204F21F330F2000130D6
:10039000F300A9204F21C830F2000130F300A9205A
:1003A0004F21F330F2000130F300A9204F216430D7
:1003B000F2000130F300A9204F21F330F2000130A8
:1003C000F300A9204F215030F2000130F300A920A2
:1003D0004F21F230F2000230F300A9204F21F33018
:1003E000F2000130F300A9204F21C830F2000130A3
:1003F000F300A9204F21F330F2000130F300A920CF
:100400004F21C830F2000130F300A9204F21F33012
:10041000F2000130F300A9204F215030F2000130EA
:10042000F300A9204F21F230F2000230F300A9209E
:100430004F21F030F2000130F300A9204F21F430B9
:10044000F2000130F300A9204F211430AB00BB01B2
:1004500083160C1583128A110A12AC2EEB30F200AF
:100460000530F300A9204F21FF30C100FF30C2004A
:1004700008086038C10006193E2A42118618412A30
:10048000C2113D1E4D2A3E08FF3C013EF10071089D
:10049000033C03184C2AC212522A3E08033C03189C
:1004A000522A4212BD1E5E2A3F08FF3C013EF10067
:1004B0007108073C03185D2AC213632A3F08073CF2
:1004C0000318632A4213BD1C662AC2103D1C692A08
:1004D0004210C01E6C2AC112401E6F2A41133D1DDE
:1004E000752ABF30C1000F30C20040080F39F1003B
:1004F000F1080319862AF11D822AFF30C1000B3052
:10050000C200862AFF30C1000730C20083160D10DA
:100510008312BB018A110A12B12E000000000000F4
:10052000000000008316051283120512000000006F
:1005300000000000000083160516831200347015B9
:10054000700883168700831207199F2A83161410D8
:100550008312AB01FF30930094132B08033C031C60
:10056000F72A83161418B62A8312B12A83121308A5
:10057000AC00941314132B08F700F7080319CD2AC5
:10058000013077020319D02A023077020319D32AE7
:10059000033077020319D62AE52A8230AD00E82A13
:1005A0005A30AD00E82A4108AD00E82A4208AD0003
:1005B0004508C23C031DE42A2C08803C031DE42AA4
:1005C0000230A8001430AB00E82A1430AD00E82A4D
:1005D0002D08930044302B0784002C0880005A30EB
:1005E0002B0784002D0880008D22AB0AAD2A8A11CA
:1005F0000A12C72E70157008831687008312071918
:10060000FA2A831614108312AB01FF30930094135F
:100610002B08073C031C722B83161418112B831212
:100620000C2B83121308AC00941314132B08F7003F
:10063000F7080319382B013077020319432B0230D6
:1006400077020319462B033077020319492B043034
:10065000770203194C2B0530770203194F2B063014
:1006600077020319522B073077020319552B602BA1
:10067000CE30AD002C08803C0319422B1430AB0067
:100680000130C300632B5A30AD00632B4108AD002D
:10069000632B4208AD00632B0130AD00632B0130AA
:1006A000AD00632B0130AD00632B0130AD00450878
:1006B000C23C031D5F2B0230A8001430AB00632B3B
:1006C0001430AD00632B2D08930044302B078400B9
:1006D0002C0880005A302B0784002D0880008D22C2
:1006E000AB0A082B8A110A12C92E02302B02FA3EDD
:1006F0000318922B063E952BC030AD00922B403054
:10070000AD00922BA908031D872BAD01892B8030EA
:10071000AD00922B4030AD00922B8030AD00922B7B
:10072000AD01922B8A110A12B02D0A148A140A11F3
:1007300082077C2B7F2B822B8A2B8D2B902B0230D8
:100740002B02FA3E0318C72B063ECA2BAD01C72B5E
:10075000AD01C72B8030AD00C72BC708031DB32BDD
:100760004030AD00B52B8030AD00C72BC708031D4E
:10077000BB2BAD01BD2B8030AD00C72BC708031DBF
:10078000C42B5030AD00C62B2830AD00C72B8A11CA
:100790000A12B22D0A148A140A118207A62BA82B5A
:1007A000AA2BAD2BB62BBE2B02302B02FA3E031820
:1007B000E92B063EEC2BAD01E92BAD01E92B4030D6
:1007C000AD00E92BAD01E92B8030AD00E92BAD0187
:1007D000E92B8A110A12B42D0A148A140A1182070D
:1007E000DB2BDD2BDF2BE22BE42BE72B02302B0264
:1007F000FA3E0318102C063E132CAD01102CAD014F
:10080000102CAD01102CC708031D092C2030AD00A1
:100810000B2CE030AD00102CAD01102CAD01102CD4
:100820008A110A12B62D0A108A100A158207FD2BAA
:10083000FF2B012C032C0C2C0E2C02302B02FA3E29
:100840000318412C063E4F2CAA08031D2A2CFF300A
:10085000AD002B2CAD01412CAA08031D322CFF301A
:10086000AD00342C8030AD00412CFF30AD00412C68
:10087000FF30AD00412CFF30AD00412CFF30AD000A
:10088000412CC708031D4B2C4808803C031D4B2CF2
:100890000130AA004C2CAA018A110A12B82D0A10A4
:1008A0008A100A158207242C2C2C352C382C3B2C32
:1008B0003E2CA908031D702C02302B02FA3E0318AF
:1008C0006F2C063E912CAD016F2CAD016F2CAD014C
:1008D0006F2CAD016F2CAD016F2CAD016F2C8E2CE8
:1008E000290B732C772C2908023C031D8E2C023017
:1008F0002B02FA3E03188E2C063E9B2CFF30AD00D7
:100900008E2CFF30AD008E2CC030AD008E2CAD0192
:100910008E2CAD018E2C5A30AD008E2C8A110A120D
:10092000BA2D0A108A100A158207632C652C672CD1
:10093000692C6B2C6D2C0A108A100A1582077E2CEC
:10094000812C842C872C892C8B2C02302B02FA3E94
:100950000318B82C063ECC2CAD01B82CAD01B82C38
:10096000AD01B82CAD01B82CAD01B82CAD01B82C3F
:10097000C708031DC92C2908FD3E0318C92C033ED6
:10098000D62CA801C92C0130A800C92C0330A8001E
:10099000C92C8A110A12BC2D0A108A100A15820766
:1009A000AC2CAE2CB02CB22CB42CB62C0A108A1065
:1009B0000A158207C12CC32CC62C02302B02FA3E2A
:1009C0000318F02C063EFE2CAD01F02CAD01F02CEE
:1009D000AD01F02CAD01F02CAD01F02CAD01F02CEF
:1009E0004708803C031DF72C0130A900FB2CC708E9
:1009F000031DFB2CA9018A110A12BE2D0A148A10AC
:100A00000A158207E42CE62CE82CEA2CEC2CEE2CC0
:100A100002302B02FA3E03181C2D063E212DAD019B
:100A20001C2DAD011C2DAD011C2DAD011C2DAD01EA
:100A30001C2D5A30AD001C2D0230A9008A110A125B
:100A4000C02D0A148A100A1582070F2D112D132D9F
:100A5000152D172D192D02302B02FA3E0318402DAB
:100A6000063E432DAD01402DAD01402D4030AD007F
:100A7000402DAD01402DAD01402D5A30AD00402D2F
:100A80008A110A12C22D0A148A100A158207322D01
:100A9000342D362D392D3B2D3D2D701570088316C4
:100AA0008700831207194D2D831614108312AB0192
:100AB000FF30930094132B08073C031CD82D83169A
:100AC0001418642D83125F2D83121308AC00941345
:100AD0001413AB08031D772DCF30AD002C08803CDC
:100AE0000319762D1430AB000130C300C92D2B0B38
:100AF0007C2D5A30AD00C92D2B08013C0318C72DA1
:100B00002B08073C031CC72D4508F700A2307702CD
:100B10000319AF2D623077020319B12DE23077024D
:100B20000319B32D323077020319B52DB230770295
:100B30000319B72D823077020319B92DC23077021D
:100B40000319BB2D223077020319BD2DF230770235
:100B50000319BF2D023077020319C12DC32D752B48
:100B6000C62D9F2BC62DD42BC62DF62BC62D1D2C86
:100B7000C62D592CC62DA52CC62DDD2CC62D082D15
:100B8000C62D2B2DC62D1430AD00C62DC92D143009
:100B9000AB002D08930044302B0784002C08800004
:100BA0005A302B0784002D0880008D22AB0A5B2D64
:100BB0008A110A12CB2E70157008831687008312D3
:100BC0000719DB2D831614108312AB01FF3093003D
:100BD00094132B08133C031C9F2E83161418F22D1C
:100BE0008312ED2D83121308AC00941314132B08F9
:100BF000F700F7080319492E013077020319542E24
:100C0000023077020319572E0330770203195A2E48
:100C10000430770203195D2E053077020319602E28
:100C2000063077020319632E073077020319662E08
:100C3000083077020319692E0930770203196B2EE9
:100C40000A30770203196D2E0B30770203196F2ECD
:100C50000C3077020319712E0D3077020319732EB1
:100C60000E3077020319752E0F3077020319772E95
:100C7000103077020319792E1130770203197B2E79
:100C80001230770203197D2E1330770203197F2E5D
:100C90008D2E9E30AD002C08803C0319532E14304D
:100CA000AB000130C300902E5A30AD00902E4208A8
:100CB000AD00902E4108AD00902E0130AD00902E79
:100CC0000130AD00902E0130AD00902E0130AD000E
:100CD000902EAD01902EAD01902EAD01902EAD0164
:100CE000902EAD01902EAD01902EAD01902EAD0154
:100CF000902EAD01902EAD01902EAD01902EAD0144
:100D00004508C23C031D8C2E4708803C031D8C2ED9
:100D10000230A8001430AB00902E1430AD00902E9D
:100D20002D08930044302B0784002C0880005A3093
:100D30002B0784002D0880008D22AB0AE92D8A1133
:100D40000A12CD2E84011F308305073083169F00C1
:100D5000FF30F000831254293B08073C031DB12EDD
:100D60002E2AC308031DCF2E2808F700F708031901
:100D7000C62E013077020319C82E023077020319FC
:100D8000CA2E033077020319CC2ECE2E9F2ACF2EE7
:100D9000FA2ACF2E4D2DCF2EDB2DCF2ECF2EAC2EDF
:020DA0006300EE
:02400E00723FFF
:00000001FF
